:020000040000FA
:020000007F2857
:020008007A2854
:02000E008A0165
:100010001708820712281F282C2839284628532819
:1000200060286D28180882074134543444343E3423
:1000300053344D3431343B340D340A340034180811
:1000400082074134543444343E3453344D343234D2
:100050003B340D340A3400341808820741345434D8
:1000600044343E3453344D3433343B340D340A3449
:100070000034180882074134543444343E34533435
:100080004D3434343B340D340A34003418088207BC
:100090004134543444343E3453344D3435343B3499
:1000A0000D340A340034180882074134543444347F
:1000B0003E3453344D3436343B340D340A3400343A
:1000C000180882074134543444343E3453344D3498
:1000D00037343B340D340A34003418088207413475
:1000E000543444343E3453344D3438343B340D347A
:1000F0000A3400340B119B0F7E2821140900031EC3
:100100008528831D85280000000083018B0183164C
:100110000F30810010308500FC308600831285018D
:100120000516970198019A019B019C019D01A1016F
:10013000A2019E019F01A001A0308B006400211C40
:10014000B528211005109C1905149C0A0F301C02BB
:10015000031CB5289C01A1142115A1159D0A02308C
:100160001D02031CB5289D0135290619061400003F
:10017000861BBC28A211C328A219C328A001A2155E
:100180002216061486148619D728A21ACC28A2167D
:10019000A0012212061086109E019F012112A112B9
:1001A00021132210A2102211851005111D29A2125F
:1001B000211AE828A11CE728A1109E0A14301E026B
:1001C000031CE6289E01211685101D2985141D2972
:1001D000061AEC282210F4282218F4282214A00170
:1001E0002117061486140000861AF828A210FC288D
:1001F000A218FC28A214A116061B00292211092905
:10020000221909292215A11A0929A001211706146A
:100210008614A11E1D29211D1D2921119F0A0A30A6
:100220001F02031C1C299F01A001A1122117051107
:100230000614861400001D290515211F3229A11D51
:100240002E29A111A00AF0302002031C2E29A001A2
:1002500021132212061D06100000312906148614EF
:1002600000009E28221E2A291F298B13061C5B29A9
:100270009A0A1F301A02031C4F299A0141306A2141
:1002800054306A2148306A210D306A210A306A21CF
:10029000970A04301702031C672997016729980100
:1002A000143099000720003E03195A296A21980A40
:1002B000990B5229672941306A2154306A2148300C
:1002C0006A210D306A210A306A2197019A01A03013
:1002D0008B00B5289100083092008511832103100E
:1002E000910C03188515031C85117D21920B6F2934
:1002F0008515832108001F3086291D3086292F305F
:100300008629103086292230862921309300930BCC
:100310008729080020342034623479343A34203478
:10032000323430343134363420345334743461341C
:100330006E346B346F34763469346334203447342C
:100340006F34723461346E34203464346934703400
:100350006C342E3469346E3467342E3465346C3426
:100360002E342034203445342D346D3461346934D6
:100370006C343A34203467346F34723461346E3400
:100380007334743461346E346B34403467346D3498
:10039000613469346C342E3463346F346D342034FA
:1003A00020342034203420342034203420342034AD
:02400E000500AB
:00000001FF
